S0160000755461736B657256312E335F424D2E7372656359
S10B200000000120494E00001C
S1132008034B1868042814BF002001207047C046F9
S1132018300100200549064B0A781A7010B9054B9F
S11320281B7801E04FF0FF330B7070472C01002040
S11320380001002038030020024B1A78024B1A7062
S11320487047C046000100202C0100207047C0469C
S1132058024A136883F0020313607047FC6302406A
S113206830B51F4B85B05A6800258DF8085092F892
S1132078213001468DF80B304FF04003ADF80430A1
S11320884FF48073ADF8063061238DF80C3092F864
S11320984B3028468DF80D3092F84C30114C8DF8A1
S11320A80E30938B6A46009303F040FB207090B186
S11320B805212A4602F08CFF009B13F0400F0AD03A
S11320C840F204412A46207802F082FF20788121D8
S11320D82A4602F07DFF034B187805B030BDC04690
S11320E8300100203803002010B5024804F0ECF950
S11320F810BDC04660680000044B012210B51A6088
S1132108612003F0F7FBFFF7EFFF10BD300100205B
S113211810B50249182203F053F810BD8068000076
S1132128182210B548F20400114904F05FFB002896
S113213813DA042018220E4904F058FB002801DBA6
S113214800240CE00A48FFF7E3FF0A4B0A499868A1
S11321583A2203F035F8002009E04FF40044054B17
S113216844F01C0099683A2204F040FB204610BD54
S113217839030020300100209868000070B5012858
S113218886B0214C20D118222049684603F018F85B
S1132198FFF7C6FF182206461C49606803F010F8CA
S11321A8A3686D461B7A13F0020F15D004A9042204
S11321B8174803F005F803A90422164803F000F8A9
S11321C8154802A9042205E0FFF7AAFF0F490646AD
S11321D86068182202F0F4FF0B4C182261680F485B
S11321E802F0EEFF60683A221830A16802F0E8FFB6
S11321F86068037E082B04D0183009493A2202F09B
S1132208DFFF304606B070BD3001002039030020DE
S11322184903002045030020410300205103002006
S113222898680000182210B548F204000C4904F01C
S1132238DDFA002809DA04201822094904F0D6FA3C
S1132248002802DA0648FFF763FF054B1A78597825
S113225842EA012242F004021A70120A5A7010BDAE
S113226839030020134B202810B518800BD002D84E
S1132278D8B1082805E0802817D0B0F5807F09D0A8
S1132288402812D014E0612041F27071062203F054
S113229853FB0DE0062261204FF4966103F04CFBDA
S11322A8054B1A78054B1A7002E0612003F022FBF3
S11322B810BDC0466A010020380300202C0100200C
S11322C810B5044B0021187802F0CCFE024B012211
S11322D81A6010BD380300203001002000B5002327
S11322E889B001930F330393E1330493094B02221A
S11322F8059306238DF81A30074B01A88DF808209A
S11323088DF809200793ADF8182002F0D3F809B026
S113231800BDC046008000203C01002070B56D4D12
S113232890B02C68867B002C40F099803A2003F00A
S113233889FAA860522003F085FA68602046FFF7FE
S11323481DFFB0F5004F08D161204FF41661032238
S113235803F0F2FA04232B6003E001232B60FFF758
S1132368C3FE00F031FA6D20042103F01DFB0320A5
S1132378FFF776FE002800F0AB80574B57481A78D1
S1132388574B1A7003F0D8F8FFF7A8FF51480123F8
S113239880F83030DB1880F836304FF00B03438672
S11323A80023C362838E643383862C3002F082F860
S11323B855E09DF8032012B1012A1AD049E09DF88E
S11323C80400032802D104F0CBF90AE0062806D158
S11323D8414B44491878162203F022F83FE0832839
S11323E802D102F02FFB3AE06C2838D1FFF776FFD0
S11323F835E09DF80430DF2B05D136490B68082BEE
S11324082DD10A602BE05E2B29D1374803F094F8CC
S1132418364803F091F80024354803F08DF800217C
S11324280A46204603F09AF8324803F085F8324BFE
S1132438822133F81400013403F086F8102CEBD110
S11324482E4803F079F8612064216C2203F074FAB1
S113245805E0304669469DF8042002F0CDFD30467B
S11324686946052202F0C8FD0028A2D1194B1B6851
S113247813F0370F2CD0184B187802F0CDFDE8B9BB
S113248826E06846214600F0A1FC1D4B1A8882B953
S11324986846214601F04EF980B14FF4807000F08F
S11324A871FD02280AD130781649172202F0B8FFC4
S11324B804E068462146002201F03CF9064E6946CC
S11324C83078402202F098FD6D4604460028D8D1A1
S11324D810B070BD3001002038030020806D00006A
S11324E82C010020D2680000A26D0000B06D00002D
S11324F8BC6D00001E7400003C01002061740000E3
S11325086A010020E968000003E09A420DD1013015
S113251801310B780278002BF7D1202A05D800E086
S113252801300378202BFBD000E000207047C04620
S113253800B5016803E003680131013303600B78D7
S1132548202BF8D04FF0000E4FF0040C10E0303B75
S1132558DAB2092A01D9D31FDAB24FEA0E139BB2B1
S113256802F00F0243EA020E0368013101330360EB
S1132578BCF1010C02D30B782F2BE8D8704600BDB0
S113258800E001300378202BFBD00F2BF9D07047E3
S11325987047C046054B31381A68C0B201238340DE
S11325A8DBB213420CBF002001207047FC630240D9
S11325B8054B31381A68C0B201238340DBB2134299
S11325C814BF002001207047006402403038642999
S11325D800B55FFA80FE0AD002D8612926D003E04C
S11325E8692904D06F290DD04FF0FF301FE0BEF1E8
S11325F8030F1BD8012202FA0EF20D48036823EADE
S1132608020309E0BEF1030F10D8012202FA0EF208
S11326180748036842EA0303064903600B681A4340
S1132628054B0A6002681B6883F84D20002000BD32
S1132638006402401C6502403401002061380F2800
S113264809D8DFE800F00A0C0E10121416181A1F25
S113265824292E33383D002036E01C4B0EE01B4B5A
S113266811E01A4B14E0194B17E0184B1AE0174BFA
S11326781DE0164B20E0154B23E0154B1B6803F0B7
S1132688010021E0124B1B68C3F340001CE0104B0F
S11326981B68C3F3800017E00D4B1B68C3F3C0002D
S11326A812E00B4B1B68C3F300100DE0084B1B68CA
S11326B8C3F3401008E0064B1B68C3F3801003E023
S11326C8034B1B68C3F3C0107047C046FC5300405B
S11326D8FC630040A0F161030F2B41D8DFE803F04D
S11326E8080A0C0E10121416181D22272C31363B1A
S11326F8224A0EE0214A11E0204A14E01F4A17E05A
S11327081E4A1AE01D4A1DE01C4A20E01B4A23E029
S11327181B4A136883F0010321E0194A136883F004
S113272802031CE0164A136883F0040317E0144AF2
S1132738136883F0080312E0114A136883F0100346
S11327480DE00F4A136883F0200308E00C4A13686D
S113275883F0400303E00A4A136883F0800313609C
S1132768084BA0F16102196801239340B1F8502085
S113277800205340A1F850307047C046FC53004035
S1132788FC6300403401002051B10B4A136843F044
S113279840031360C03A136823F04003136002E057
S11327A8064B1B681840064B18601A68054B1B68D3
S11327B883F84E207047C04608E10F400064024089
S11327C8FC6302403401002070B5934901250A686E
S11327D892F84E3092F84D6006EA030382F84E30C0
S11327E80B68012193F84E00FFF7CEFF30203542E5
S11327F800F10103DCB214BF6F216921FFF7E6FE83
S1132808382C03D06B00DDB22046F0E7834B01215E
S11328181A68002042F006021A607F4B1D68B5F85A
S11328285040214268D080293CD010D8082931D0A2
S113283806D802292AD004292AD0012924D0C4E0A0
S113284820292BD040292BD0102925D0BDE0B1F563
S1132858006F38D009D8B1F5007F2AD0B1F5806F60
S11328682CD0B1F5807F1FD0AFE0B1F5005F34D034
S113287803D8B1F5805F2BD0A7E0B1F5804F31D0F4
S1132888B1F5004F33D0A0E0654A0EE0644A11E088
S1132898634A14E0624A17E0614A1AE0604A1DE09C
S11328A85F4A20E05E4A23E05E4A136843F001036E
S11328B88AE05C4A136843F0020385E0594A1368C6
S11328C843F0040380E0574A136843F008037BE0AD
S11328D8544A136843F0100376E0524A136843F0ED
S11328E8200371E04F4A136843F040036CE04D4AFB
S11328F8136843F0800367E080293CD010D8082986
S113290831D006D802292AD004292AD0012924D072
S11329185BE020292BD040292BD0102925D054E066
S1132928B1F5006F38D009D8B1F5007F2AD0B1F5D8
S1132938806F2CD0B1F5807F1FD046E0B1F5005FE1
S113294834D003D8B1F5805F2BD03EE0B1F5804F89
S113295831D0B1F5004F33D037E0314A0EE0304A78
S113296811E02F4A14E02E4A17E02D4A1AE02C4AA7
S11329781DE02B4A20E02A4A23E02A4A136823F060
S1132988010321E0274A136823F002031CE0254AC7
S1132998136823F0040317E0224A136823F008039A
S11329A812E0204A136823F010030DE01D4A13684F
S11329B823F0200308E01B4A136823F0400303E0D4
S11329C8184A136823F08003136001304B00102861
S11329D899B27FF426AFA5F850406122531CD9B2AE
S11329E8A2F161030F2B7BD8DFE803F0080A0C0E71
S11329F810121420222D38434E59646F0A4A18E0E5
S1132A08094A21E0084A2AE0074A33E0064A3CE03A
S1132A18054A45E0044A4EE03401002008E10F402D
S1132A28FC530040FC6300401C5500402F4A4DE015
S1132A382F4A136843F001031360A2F58E721368DA
S1132A4843F001034BE02A4A136843F0020313607E
S1132A58A2F58E72136843F0020340E0244A136817
S1132A6843F004031360A2F58E72136843F0040361
S1132A7835E01F4A136843F008031360A2F58E7209
S1132A88136843F008032AE0194A136843F0100353
S1132A981360A2F58E72136843F010031FE0144A02
S1132AA8136843F020031360A2F58E72136843F091
S1132AB8200314E00E4A136843F040031360A2F5A0
S1132AC88E72136843F0400309E0094A136843F01F
S1132AD880031360A2F58E72136843F080031360B9
S1132AE8712901D00A4679E770BDC0461C550040DB
S1132AF81C6500407047C0460020704770B500E070
S1132B0801310B782B2BFBD0042817D0072829D0A8
S1132B1803282DD1174D08462C6802F03BFB84F896
S1132B284B002D6895F84B30632B01D9632302E0E1
S1132B38092B1DD80A2385F84B3019E00D4D08469A
S1132B482C6802F027FB84F84C002D6895F84C306B
S1132B58632B01D9632302E0092B09D80A2385F8DA
S1132B684C3005E0034B08461C6802F013FBE08375
S1132B7870BDC0463401002070B50F4B0246196879
S1132B888B78CC78487904EB03248B79CD790004CD
S1132B9800EB03200B794019022100EB036002F0DB
S1132BA8DDFCA4B202462D2302F8013B2046022193
S1132BB802F0D4FC70BDC04634010020204B2DE93E
S1132BC8F0411C681F4D1423B4FBF3F4B4FBF5F86F
S1132BD802460021404602F0C1FC2026024602F8C3
S1132BE8016B08FB154544234370511C1D33537076
S1132BF8481C18334B70421C73234FF461644370B0
S1132C085670B5FBF4F600210232304602F0A6FCF9
S1132C1806FB14543C2602464FF03A08B4FBF6F57A
S1132C2802F8018B0221284602F098FC024602F8B9
S1132C38018B05FB1640022102F090FCBDE8F081EF
S1132C486C0300208051010010B5084C2068FFF780
S1132C585FFA206806220230054902F0B1FA2068BA
S1132C68044918303A2202F0ABFA10BD34010020AE
S1132C783B03002098680000022870B5054611D16E
S1132C88174B1868174B90F820201B6802F00202B3
S1132C981B7A03F002039A4220D11349182202F046
S1132CA89DFAD8B90E4C1822216848F2040003F0A2
S1132CB879FD21683A22183148F21C0003F072FDAC
S1132CC8012D09D0022003F04BFD2168054B183172
S1132CD818683A2202F074FA002000E0012070BD5E
S1132CE8340100203801002051030020204B10B586
S1132CF81868204B828B19688B889A4212D190F8F5
S1132D084B2091F833309A420CD190F84C2091F82A
S1132D1834309A4206D190F821204B7AD41A18BF3D
S1132D28012400E0012490F82000097A00F0280228
S1132D3801F028039A4200F0040201F0040318BFCA
S1132D4844F002049A4200F0100201F0100318BF84
S1132D5844F004049A4218BF44F008040120FFF721
S1132D680DFA14F0010F02D00420FFF779F910BD11
S1132D7834010020380100202DE9F041124B0125CF
S1132D881B68312093F84D70B3F850800026431C1B
S1132D98DCB2FFF7FFFB00B12E43392C03D06B00E4
S1132DA8DDB22046F3E7FFF7A1FF074A00201368C6
S1132DB883F84D70136883F84E601368A3F8508045
S1132DC8FFF75AFFBDE8F0813401002010B50A4628
S1132DD8034903460878194602F022FB10BDC04691
S1132DE83803002010B50C4602F0A6FB094802F08F
S1132DF8A3FB094B1B6893F820301C4004D00748F8
S1132E0802F09AFB012003E0054802F095FB2046F6
S1132E1810BDC04684710000340100208871000090
S1132E289271000002281FB502D004281FD024E0A4
S1132E38124802F081FB6846FFF79EFE684602F0DE
S1132E487BFB0F4802F078FB0E4802F075FB0E4836
S1132E5802F072FB0A4802F06FFB0C4802F06CFBAC
S1132E680B4B6C461868363002F066FB05E0084BDD
S1132E7814221868363002F0A3F91FBD9D710000B2
S1132E88DA710000AF710000397B0000C1710000E5
S1132E98340100202DE9F04FDFF8E4A04FF00C09CD
S1132EA89AF80030314D03FB09F35A19547989B063
S1132EB8804692F804B00DF1050020211B225E59CA
S1132EC8274602F075F9B8F1000F07D0002301E096
S1132ED80C360133FC1A4445FADC3EE0244802F07F
S1132EE82BFB9AF8003003FB0953986802F024FB83
S1132EF8204802F021FB30E06B88013C202B03D0F2
S1132F08AB88B3F5805F10D11B4F0021387842227B
S1132F1802F086FA48B93878402141F26D0202F08D
S1132F2857F8631CAB6001201CE0306802F004FB16
S1132F3858450DF10501104B02DB1878012203E016
S1132F48C0EB0B02187892B202F06AFA706802F0C9
S1132F58F3FA0A4802F0F0FA0C36094D002CCBD1EA
S1132F68AC60204609B0BDE8F08FC046D46D0000BF
S1132F78D9710000DD7100002C010020DA71000015
S1132F8868010020B0F5807F70B5104A06D1938897
S1132F98D3B99389C3B9FFF765F902E04FF4007315
S1132FA893810A4D6B88B3F5807F02D12020FFF707
S1132FB859F9002402200021FFF734FF20462C7021
S1132FC8FFF768FF204600E0022070BD680100207A
S1132FD870B504460D461148214602F013F901461E
S1132FE850B121460E4802F00DF9014658B10D487A
S1132FF802F0A2FA01200FE00B4B1A6892F8203075
S113300845EA030305E0084B1A6892F8203023EADE
S1133018050382F82030084670BDC046F5710000EB
S1133028FC7100000472000034010020F0B50C4665
S113303889B01546072800F25583DFE810F0080028
S11330482B00E900050153039A010403090309B994
S1133058084605E0042906D10122934B00201A7082
S1133068FFF718FF3FE3052901D10222F5E70629F6
S113307801D10322F1E7072901D10422EDE7092947
S113308801D10522E9E70D2940F02C83864B002065
S11330981870E5E70C2900F22583DFE811F00D002C
S11330A810009500230380004B002303230323030C
S11330B823032D0038007D0001F0C4FC12E37B4893
S11330C802F03AFA7A4802F037FA7A4802F034FA07
S11330D802F08EFB822102F037FA774802F02CFACC
S11330E802F07EFB822102F02FFA744802F024FADF
S11330F802F06AFB822111E101AD2846FFF75EFD6B
S1133108002404706E4802F017FA284659E0137830
S1133118313BDBB2032B01D96A48E1E26A4802F089
S11331280BFA2878FFF744FA044608B9674848E0D8
S11331386748D5E21078A0F13103DBB2032B33D80A
S1133148FFF736FA08B16348CAE207460126312078
S1133158431CDCB2FFF71EFA10B146EA0703DFB2DC
S1133168352C03D07300DEB22046F1E7284601F07F
S1133178FBFFC0B2013801238340681CDCB201F0B4
S1133188F3FF01280CBF44EA070327EA0403D8B273
S11331980021FFF7F9FAA5E2FFF7EEFDA2E21378A2
S11331A8313BDBB2032B01D94B4899E24B4802F07F
S11331B8C3F92878FFF7EEF9044608B148488FE2C6
S11331C8484802F0B9F93DE0104601F0CDFF2B78EC
S11331D80246202B01D0284604E0284609E0202B8B
S11331E807D001300378002BF9D102E0202904D15B
S11331F8013001780029F9D108E039B102F12F0032
S1133208C0B2FFF7E3F9002800F06C82364867E2A1
S113321849B1032940F06682344B10461C6801F01A
S1133228B9FFE0835EE2204DAB89042B06D1304818
S113323802F082F94FF01003AB8103E0A98008463D
S1133248FFF710F820464EE20692072900F24A8258
S1133258DFE801F00454798015858A6A06AC2046B3
S1133268FFF766F905462046FFF762F908A901F851
S1133278010D0122284603F095FA1E4830E206ACF7
S11332882046FFF755F905462046FFF751F96FEA3E
S1133298454508A96FEA554501F8010D0122A8B270
S11332A803F080FA14481BE268010020177200003A
S11332B8E07100002E7200003B72000042720000B0
S11332C854720000797200008B7200009E72000034
S11332D8A7720000BE720000AF720000CE72000038
S11332E8DB720000DF720000E3720000340100208A
S11332F8EB720000F77200000973000006A8FFF7DC
S113330817F901220DF11F0103F070FA002809DBF7
S1133318914802F011F99DF81F00012102F014F9F7
S11333288E48DDE18E48DBE18E4C8F4918222068F7
S113333801F046FF20688D4B183019683A2201F0D5
S11333483FFF8B48CCE1FFF77FFC0020FFF794FC9C
S11333588848C5E1012003F003FA8748C0E1022048
S113336803F0FEF98548BBE10020FFF785FC84489B
S1133378B6E1162900F2B681DFE811F017005A0009
S113338828003C007A00B401B401B401B401B401CA
S1133398B401B401B401B401B401B401B401990095
S11333A8B401B401B4014D014D016E4B754E1F6853
S11333B800243046294601F025FF10B987F821403A
S11333C83DE1013407360C2CF3D182E1107837281B
S11333D805D1644B1A68938B43F0010306E038283F
S11333E806D1604B1A68938B23F00103938326E17B
S11333F8654875E15B4B654F1C68002638462946CD
S113340801F000FF78B9A38B4FF6F97203EA0202C0
S1133418A28316B1012E03D011E142F004031DE08A
S113342842F002031AE001360537032EE6D152E1D1
S11334384C4B574E1C6800273046294601F0E2FEE3
S113344888B9A38B4FF6E77203EA0202012FA2831D
S113345802D0022F04D0F2E042F00803A383EEE086
S113346842F01003FAE701370436032FE4D134E1BC
S11334783C4B484E1C6800273046294601F0C2FEE2
S113348880B9A38B4FF69F7203EA0202012FA2832D
S113349802D0022F03D0D2E042F04003DEE742F02C
S11334A82003DBE701370836032FE5D117E13A4853
S11334B802F042F8394802F03FF82A4B1B6893F8A7
S11334C821200B2A04D82F48072302FB030000E01D
S11334D8334802F031F8334802F02EF8214B1B68C8
S11334E89B8B13F0010F14BF2F48304802F024F8C7
S11334F82F4802F021F81B4B1B689B8B13F0020F1B
S113350801D0012204E013F0040F0CBF02220022B0
S11335181E48052302FB030002F00EF8254802F0BA
S11335280BF8104B1B689B8B13F0100F01D0022370
S113353801E0C3F3C003164800EB830001F0FCFF6D
S11335481D4801F0F9FF074B1B689B8B13F0400FD4
S113355834D0012437E0C04621730000DA7100003A
S1133568367300003401002039030020380100209C
S1133578587300007973000099730000B473000055
S1133588D17300001C6E0000E9730000706E000027
S11335987F6E00008B6E0000017400001A74000036
S11335A822740000617400002B7400002D74000064
S11335B82F740000E27400003774000013F0200335
S11335C80CBF1C460224494801F0B6FF484800EBEA
S11335D8C40001F0B1FF474801F0AEFF002C00F031
S11335E88180454C454801F0A7FF236800210A461D
S11335F893F84B0001F0B2FF414801F09DFF4148A8
S113360801F09AFF2368002193F84C000A4601F060
S1133618A5FF3B4864E0104601F0BCFDC0B2632836
S113362801D9632002E0002808BF0120324B152C81
S11336380BBF1B681B6883F84B0083F84C000420FD
S1133648FEF70EFD4EE008461146FFF7EBFB49E096
S1133658062947D8DFE801F004070C1218150F00F3
S11336681046102101E010460221FFF7B1FC39E0B1
S113367810460421F9E710464021F6E710460821D0
S1133688F3E710462021F0E71F4801F055FF4021D9
S11336981E48FFF7A7FB04211D48FFF7A3FB1D489D
S11336A80821FFF79FFB18B11B482021FFF79AFB5D
S11336B81A481021FFF796FBA0B1194801F03CFF06
S11336C80D4B00211B680A46D88B01F047FF0948B7
S11336D806E0144804E0144802E0144800E01448E2
S11336E801F02AFF002009B0F0BDC046467400006E
S11336F88B6E0000617400003401002054740000D3
S113370860740000647400006F7400008574000025
S1133718D2790000217A00004A7A000099740000E6
S1133728A7740000C0740000D9740000EC74000091
S1133738027500002DE9F0478046894617460025A2
S11337487DE098F80030082B09D1434A937B002B7D
S113375875D0013B9373414801F0EEFE6FE00A2BEC
S11337686DD0002B6BD03C4CA27B1119CB7398F80D
S113377800300D2B59D10A23CB733846FEF74AFC87
S1133788A37B0C220133D8B22378354903FB02F317
S11337985A185D585179002304F10E0213542FB9B5
S11337A86288002A3AD012F4806F37D1002832D0C8
S11337B80C4613E0284E296806F10F00FEF7A4FE14
S11337C8024650B1287A697AFFF730FC10B92548C7
S11337D801F0B2FE17BB708816E00C35013CE9D243
S11337E8214C15E01C4D216805F10F00FEF78CFEF5
S11337F8024660B1207A617AFFF718FC10B91948BB
S113380801F09AFE57B96888FEF72CFD06E00C34DF
S1133818164B9C42E6D1164801F08EFEFEF70CFCCE
S11338280D4B00229A73012501E0531CA3730A4A25
S113383808F10108937B272B01D92723937309F1F6
S1133848FF331FFA83F94FF6FF7399457FF479AF75
S11338582846BDE8F087C04668010020A46E000031
S1133868D46D0000E7720000A86E0000B46E00007A
S1133878E372000030B589B0847B32E09DF80330F0
S1133888012B02D0412B14D025E09DF80430DF2B06
S113389827D1194A906810B1FFF7FCFA21E092F891
S11338A8373013F0010F1CD023F0010382F83730AE
S11338B817E0204669469DF8042001F09DFB9DF819
S11338C80030042B01D10D4802E0032B09D10C4828
S11338D801F032FE05E0204669469DF8042001F017
S11338E88BFB2046694605226D4601F085FB0028BE
S11338F8C4D109B030BDC046680100201B75000062
S11339082C7500000C4B00B543F820200B4A2023EB
S113391800EA0202002A90FBF3FE05DA013A6FEA94
S1133928C2626FEAD262013201239340044A42F828
S11339382E30044BC15400BD400000201F000080FD
S113394800E100E000E400E0044B00221A60044AAD
S1133958136883F0040313607047C0460C000040EA
S1133968FC63024072B6024A13680133136070475D
S1133978A0010020034A1368013B136003B962B62F
S11339887047C046A0010020074A084B1A60084A3D
S11339984FF00053DA63074A136843F0E063136097
S11339A8054B07221A6070479F25260014E000E0A3
S11339B80D4E000020ED00E010E000E0072807D8D5
S11339C8DFE800F0080A0C0E1012140408480EE090
S11339D800200CE007480AE0074808E0074806E02A
S11339E8074804E0074802E0074800E00748704732
S11339F8FC730240FC430040FC530040FC6300405D
S1133A08FC730040FC430240FC530240FC63024048
S1133A18012808D005D3054B02280CBF18460020FE
S1133A2802E0034800E003487047C04600E0004055
S1133A3800C0004000D00040012810B507D002D3D0
S1133A48022808D00CE005200621064A06E00620D4
S1133A580146054A02E0054A21200621FFF752FFE4
S1133A6810BDC046C94D0000854D0000414D000001
S1133A7870B50546FFF7CCFF04462846FFF7DCFF80
S1133A8810236364A36B43F01003A363236B43F411
S1133A980073236370BDC04610B5FFF7B9FF836B8D
S1133AA823F010038363036B23F40073036310BDD3
S1133AB870B50546FFF7ACFF04462846FFF7BCFF80
S1133AC820236364A36B43F02003A363236B43F4B1
S1133AD88073236370BDC04610B5FFF799FF836BED
S1133AE823F020038363036B23F48073036310BD03
S1133AF87047C04610B50C46FFF78AFF836913F078
S1133B08800F01D1012001E00460002010BDC046EF
S1133B1810B101280BD015E021B10B4A136823F02A
S1133B2802030EE0084A136843F0020309E021B1D6
S1133B38054A136823F0010303E0034A136843F0BA
S1133B48010313607047C046FC73004011F4C05F62
S1133B5870B504460D4663D011F4006F27D010B138
S1133B68012810D01FE0374A136843F00803136094
S1133B78354A136843F002031360A2F58E72136882
S1133B8843F002030EE02F4A136843F0080313605E
S1133B982D4A136843F001031360A2F58E7213686B
S1133BA843F00103136020460021FFF7B1FF15F429
S1133BB8805F35D0012C13D002D3022C20D02FE003
S1133BC8204A136843F001031360204A136843F042
S1133BD808031360A2F58E72136823F008031EE02D
S1133BE8184A136843F001031360184A136843F032
S1133BF880031360A2F58E72136823F080030EE02D
S1133C08104A136843F001031360104A136843F021
S1133C1840031360A2F58E72136823F04003136007
S1133C2840F2011105EA010111B12046012105E024
S1133C3840F2022305EA030313B12046FFF768FFA5
S1133C4870BDC04608E10F401C7500401C4500408B
S1133C5870B505460E46FFF7DBFE0023012D04462A
S1133C6803631DD002D3022D3CD05DE05F4A136884
S1133C7843F001031360C03A136823F0010313608F
S1133C88136823F001031360BC32136843F0010383
S1133C981360C03A136823F001031360544A3AE0EE
S1133CA8524A136843F008031360C03A136823F0B8
S1133CB808031360136823F008031360BC32136805
S1133CC843F002031360C03A136823F0020313603D
S1133CD8484A136843F00C031360FC32136843F03A
S1133CE80C0320E0414A136843F040031360C03AD0
S1133CF8136823F040031360136823F04003136030
S1133D08BC32136843F004031360C03A136823F009
S1133D1804031360384A136843F003031360FC3246
S1133D28136843F003031360336813F0400F05D09E
S1133D3828464FF4C0510022FFF708FFF37A0B2BF3
S1133D4828D8DFE803F00C1014181C2024272A2D87
S1133D5806091B22082325E00D22242322E042F62B
S1133D68B0022B231EE041F2584215231AE040F614
S1133D782C220B2316E040F21652052312E040F2DF
S1133D888B2203230EE040F2451221230AE0D922B4
S1133D98012307E0A222312304E05122182301E081
S1133DA8362210236262A362336813F0060207D036
S1133DB813F0040F01D0022300E00623E36200E0BD
S1133DC8E262336813F0100F03D0E36A43F0080388
S1133DD8E362336813F0010FE36A14BF43F040034E
S1133DE843F06003E3620123236370BD08E10F40DD
S1133DF8204400402074004020640240074B1A60AD
S1133E08043B1960064A40F0244343F484031360D6
S1133E18034B1B681842FBD17047C04604D00F40BF
S1133E2808D00F4070B520F47E740D4624F00704C2
S1133E38084B002602201E6021463246FFF7DEFFAB
S1133E48B5F5806F04D904F58064A5F58065EFE7BE
S1133E58304670BD0C00004070B520F003040E46D7
S1133E68154600F00300236817E0C100FF228A40CA
S1133E7823EA02023378013D8B40032842EA030314
S1133E8809D1012021461A46FFF7B8FF65B154F855
S1133E98043F002000E001300136002DE5D1012067
S1133EA821461A46FFF7AAFF002070BD10B54FF44B
S1133EB80061FFF7B7FF10BD2DE9F3411C465523F8
S1133EC810F0800F0F4690468DF8073001D1002678
S1133ED802E000F07F00012610F0400F0AD04FF4F2
S1133EE8C030FFF7E3FF4FF4C430FFF7DFFF4FF4B0
S1133EF8C03505E0022814BF4FF4C0354FF4C4356B
S1133F0884B956B1B5F5C03F14BF4FF4C0304FF46F
S1133F18C430FFF7CBFF26460AE02846FFF7C6FF62
S1133F289FB905E0E819023041462246FFF794FF9D
S1133F380DF10704284621460122FFF78DFF26B913
S1133F48681C21460122FFF787FF0020BDE8FC8199
S1133F5828B1044B01280CBF1846002000E0024891
S1133F687047C046001002400000024070B5C47992
S1133F7806462046FFF7ECFF0546002C2DD1364AAD
S1133F8808201368042143F002031360C03A13683D
S1133F9823F002031360136823F002031360BC3296
S1133FA8136843F480531360C03A136823F48053AE
S1133FB813602A4A136843F00C031360FC32136835
S1133FC843F00C031360103A136843F00C031360B6
S1133FD8234B01221A60234A2CE01F4A2520136828
S1133FE8042143F001031360C03A136823F001036A
S1133FF81360136823F001031360BC32136843F49D
S113400880431360C03A136823F480431360164A4C
S1134018136843F0C0031360FC32136843F0C00311
S11340281360103A136843F0C00313600F4B012266
S11340381A600F4AFFF766FC3088102332282B6277
S113404806D0B0F5C87F01D1052302E0182300E0AB
S11340583123EB6070BDC04608E10F402054004096
S11340681C0002402D4C0000204400401C1002405B
S11340780D4C000070B5044608460D46FFF768FF6E
S1134088636813F8012BA275E2686360934224BF46
S113409823686360636813F8012B0260E268636055
S11340A8934224BF23686360036813F0010F1AD096
S11340B8A37D012B01D1063300E00B2343606FF08D
S11340C83F03E375238A6268033B2382154B53F845
S11340D8251012F8013B0B76E36862609A4220D3FC
S11340E8236863601DE0636813F8012B82606360D2
S11340F8A37D012B01D1063300E003234360012390
S113410803616268E3689A4228BF2368A27D28BFD6
S113411863604023E375238A9B1A013B013A238297
S1134128A27570BD2403002070B50C4D80240FE0E7
S113413813681C4207D00A4B1C60FFF713FCEB6999
S11341489847FFF717FC074B043D64089D4203D0CA
S1134158054A1368002BEBD170BDC046A4010020AA
S11341681C440040840100201844004070B50D4CE4
S1134178802511E013681D4209D00B4B1D60E369CB
S11341882BB1FFF7EFFBE3699847FFF7F3FB074B06
S1134198043C6D089C4203D0054A1368002BE9D1FE
S11341A870BDC046C40100201C540040A401002076
S11341B81854004070B50C4D80240FE013681C425D
S11341C807D00A4B1C60FFF7CDFBEB699847FFF754
S11341D8D1FB074B043D64089D4203D0054A13688C
S11341E8002BEBD170BDC046E40100201C640040E4
S11341F8C40100201864004070B50C4D80240FE001
S113420813681C4207D00A4B1C60FFF7ABFBEB6931
S11342189847FFF7AFFB074B043D64089D4203D062
S1134228054A1368002BEBD170BDC0460402002078
S11342381C740040E40100201874004070B50C4D53
S113424880240FE013681C4207D00A4B1C60FFF758
S113425889FBEB699847FFF78DFB074B043D64081E
S11342689D4203D0054A1368002BEBD170BDC046AC
S1134278240200201C440240040200201844024086
S113428870B50C4D80240FE013681C4207D00A4B0C
S11342981C60FFF767FBEB699847FFF76BFB074B5D
S11342A8043D64089D4203D0054A1368002BEBD1F2
S11342B870BDC046440200201C5402402402002061
S11342C81854024070B50C4D80240FE013681C424A
S11342D807D00A4B1C60FFF745FBEB699847FFF7CB
S11342E849FB074B043D64089D4203D0054A136803
S11342F8002BEBD170BDC046640200201C64024050
S1134308440200201864024070B50C4D80240FE06C
S113431813681C4207D00A4B1C60FFF723FBEB69A8
S11343289847FFF727FB074B043D64089D4203D0D9
S1134338054A1368002BEBD170BDC04684020020E7
S11343481C740240640200201874024070B50C4DBD
S113435880240FE013681C4207D00A4B1C60FFF747
S113436801FBEB699847FFF705FB074B043D64081D
S11343789D4203D0054A1368002BEBD170BDC0469B
S1134388A40200201CD403408402002018D4034053
S1134398064B01221A6010B5FFF7E4FA044BD3F870
S11343A824319847FFF7E6FA10BDC04624000340BD
S11343B8A0010020064B01221A6010B5FFF7D2FABB
S11343C8044BD3F828319847FFF7D4FA10BDC046F8
S11343D824100340A0010020064B01221A6010B5E6
S11343E8FFF7C0FA044BD3F82C319847FFF7C2FA09
S11343F810BDC04624200340A0010020064B012222
S11344081A6010B5FFF7AEFA044BD3F83031984769
S1134418FFF7B0FA10BDC04624300340A0010020C5
S11344281D4A012313601D4B10B5D3F83421002015
S113443805E022B11A4B01301B6822F8023B194BE4
S11344481B6813F4807FF4D0144CB4F83811C4F802
S1134458342101290CD8144A136823F480331360D7
S113446801232360D4F83C3198470023236012E0E9
S1134478D4F83C311BB14B1EA4F8383103E0A2EB4D
S11344884003C4F83431094B1B6813F00F0F02D1F1
S1134498074B01221A6010BD0C800340A0010020C4
S11344A8488003404C80034000E10F4014800340DF
S11344B8288003402DE9FF4703790546012B00F0C6
S11344C8DD8003D3022B00F0288157E2C27901234F
S11344D89340DFB2002F00F051828079082800F25F
S11344E84D82DFE800F0050E172029323B444D00C9
S11344F8944B4FF0000A03EB82080126DFF89092F0
S113450847E0914B4FF0010A03EB82080226DFF8DB
S113451884923EE08D4B4FF0020A03EB8208042696
S1134528DFF8749235E08A4B4FF0030A03EB8208F4
S11345380826DFF868922CE0864B4FF0040A03EB58
S113454882081026DFF8589223E0834B4FF01E0AA6
S113455803EB82082026DFF84C921AE07F4B4FF0D9
S11345681F0A03EB82084026DFF83C9211E07C4BDB
S11345784FF0200A03EB82088026DFF8309208E027
S1134588784BDFF82C9203EB82084FF0360A4FF48D
S11345988076FFF713FA2B68044663B96B7A082B05
S11345A809D0436923EA07034361002B40F0E681FD
S11345B802226D4BE1E16D4AF943136846EA0303AD
S11345C81360C03A136823EA06031360636AA26897
S11345D80B406362636801EA03036360D4F8203123
S11345E83B43C4F820312B7A012B10D902EA01038A
S11345F8A3602B7A042BE36802D13B43E36015E004
S11346080B40E3602B7A2269032B09D00BE0E368A3
S11346180B40E36042EA0703A3602B7A226913B9CB
S113462842EA070301E002EA010323616B7A022BE1
S113463809D0082B0CD0012B13D1D4F814313B43E7
S1134648C4F814310DE0D4F818313B43C4F81831D8
S1134658474B1B6813F0020F0CD1464B10221A600B
S113466808E02762504669794A46FFF74BF92B68F8
S1134678C8F8003063693B4363617FE1867A032E9F
S113468800F37C814FF4803202FA06FE3A493B4A31
S11346980B684EEA03030B604FEA063303F18044C8
S11346A8136804F540344EEA0303136001D1232050
S11346B802E0730003F113002F4A136823EA0E0380
S11346C813602B6863B12E4B697953F82620FFF7E2
S11346D819F92C4B2A6803EB8603C3F82421012318
S11346E8A361EB8813F0020F01D0022300E0012339
S11346F86360EB882A8913F0010F14BF4CF250331E
S1134708322302FB03F3A362EB8813F0080F01D0F2
S1134718212300E00123E36030E1036913F4801FDF
S113472808D0194B00221A60184A136823F48033FE
S1134738136023E113F4804F48D08169002945D0E0
S1134748828A3EE0A4010020C4010020E401002084
S113475804020020240200204402002064020020F5
S113476884020020A402002080E100E008E10F4058
S113477800E100E01C54004044E00F4004E10F4015
S1134788447B0000A00100200880034000E10F40A2
S11347983141000075410000BD41000001420000A4
S11347A84542000089420000CD4200001143000048
S11347B855430000724B1B681AB121F8023B531E83
S11347C89AB2704B1B6813F4807FF3D0296911F4F3
S11347D8805440F0D38011F4004F00F0C8806A4A36
S11347E86A48136843F480331360694AD5F80C8027
S11347F81368D5F8089023F001031360036823F0C5
S11348080F02644B026001EA0303002B67D011F422
S1134818403F2AD02B698DF8084003F44033B3F5A0
S1134828003F019407D0B3F5403F06D0B3F5803F6D
S113483806D1032302E0022300E004238DF80C30A0
S113484801238DF80A30DB188DF8093002338DF80E
S11348580B3001A804338DF80D30FFF72BFE4B4ABB
S1134868136843F0040313603AE011F0404311D095
S1134878B3F1004F08D0B3F1404F08D0B3F1804FE3
S11348882ED142F0010328E042F0020325E042F071
S1134898030322E011F0005F02D042F005031CE09C
S11348A811F048631CD0B3F1806F0ED003D8B3F570
S11348B8000F07D014E0B3F1006F09D0B3F1406FD3
S11348C809D00DE042F0060307E042F0070304E0D4
S11348D842F0080301E042F00903036000E00260CB
S11348E8AA7D2D4B00201A6001460746044601267E
S11348F849EA08031E4212D016EA080F0AD014F037
S1134908010F0CD18B0001229A40174362089A4088
S1134918104303E08B0014FA03F3184301317600C3
S1134928072C01D00134E3E741B34B1E9B00062258
S11349389A401A4B3A43186004331A600E20184AF6
S11349486979FEF7DFFF174A2B68C2F83C31AB8A56
S1134958A2F83831AB69C2F83431134A136843F00A
S113496801031360083A136843F0010313602B69C9
S113497813F0100F02D00D4B01221A60BDE8FF8717
S1134988488003404C80034000E10F4014800340FA
S113499800800340000083EC3080034040800340E3
S11349A829440000A0010020088003402880034017
S11349B830B511F00C0F85B0054627D000238DF8CB
S11349C8083011F0040303D01C4B03EB80031B696C
S11349D801931A4BEB181A7FDC7F93F822008DF8A9
S11349E80A200022D1B24B1C013250FA03F3F9D148
S11349F801238DF80D3003330DEB03008DF80940C6
S1134A088DF80B108DF80C30FFF754FD0C4B1A6819
S1134A180A4BEC18207F0123834013420AD0FEF787
S1134A28CDFF38B1026894F82230134202D14FF412
S1134A38807000E0002005B030BDC046447B000013
S1134A4808E10F40084A136843F008031360074A53
S1134A58074B1A600022A3F540631A60054A022333
S1134A68136001331360FEE700E10F4051E5CC1AEF
S1134A78000C0040080000407047C0467047C0461C
S1134A887047C0467047C0467047C0467047C04626
S1134A987047C0467047C0467047C046052300FBB0
S1134AA803F082B00190019A531E0193002AFAD1AF
S1134AB802B07047114A124BD01A002104E0114B7E
S1134AC8CA5C0F4BCA5401318142F8D10E4A0F4BCC
S1134AD80021D01A04E00E4BCA5C0C4BCA540131B5
S1134AE88142F8D10B4A0C4B0021D01A03E00A4B3F
S1134AF80022CA5401318142F9D170472D010020A6
S1134B0800010020F47B0000606800000820000019
S1134B18082000007803002030010020D0F800D0DD
S1134B28D0F804F07047C0462DE9F04192F91730E7
S1134B388046002B0E461446957D35DA304FDDB19C
S1134B486B1E937557F82010B2688B6803F8012B15
S1134B588B60A37D0BB9053300E009237360284BF0
S1134B6853F82800038A826801330382C3689A428F
S1134B7844D30368836041E057F820309A8A0132AD
S1134B889A8293F9183053B1FEF7ECFE57F828309F
S1134B98042193F9180000F007FFFEF7EBFE238ABF
S1134BA843BB3561E57529E09DB16B1E9375536868
S1134BB813F8012B8A606360A37D0BB9053300E009
S1134BC8012373606268E3689A4217D323686360B9
S1134BD814E0138A73B90B61D37592F918306BB169
S1134BE8FEF7C0FE94F91800042100F0DDFEFEF77C
S1134BF8C1FE03E020464146FFF73CFABDE8F081D8
S1134C0824030020044B01201860044B10B5044908
S1134C185A68FFF789FF10BD1C100240700300207A
S1134C2800100240054A01231360054B10B500200B
S1134C3804491A68FFF778FF10BDC0461C000240FB
S1134C487003002000000240034610B508461946C8
S1134C5800F0B6FA10BDC046022814BF4FF4C030A5
S1134C684FF4C430401870B51E46851C07E0541C28
S1134C78284611460122FFF7E7FF01352246731E35
S1134C889EB24FF6FF739E42F1D1002070BDC0461C
S1134C9813B5022204460DF106014FF4C030FFF7A4
S1134CA8D3FF9DF80630002C0CBFFF245524552B48
S1134CB805D19DF80730A34201D1012011E0022259
S1134CC84FF4C4300DF10601FFF7BEFF9DF806301E
S1134CD8552B05D19DF80730A34201D1022000E0ED
S1134CE800201CBD10B50020FEF768FE01680220F4
S1134CF881F04001C1F3801100F0FAFF10BDC046F5
S1134D0810B50020FEF75AFE0168012081F08001E9
S1134D18C1F3C01100F0ECFF10BDC04610B500206F
S1134D28FEF74CFE0168002081F00801C1F3C001C0
S1134D3800F0DEFF10BDC04610B516E0236813F07E
S1134D48100F08D00B4B10221A60443B186802213C
S1134D58C0B200F0E5FF236813F0200F05D0054B1F
S1134D6820221A60022000F0B9FF034C2368002BAC
S1134D78E4D110BD44E0004040E0004010B516E026
S1134D88236813F0100F08D00B4B10221A60443B11
S1134D9818680121C0B200F0C3FF236813F0200F84
S1134DA805D0054B20221A60012000F097FF034C20
S1134DB82368002BE4D110BD44D0004040D000400B
S1134DC810B516E0236813F0100F08D00B4B10220F
S1134DD81A60443B18680021C0B200F0A1FF2368A0
S1134DE813F0200F05D0054B20221A60002000F094
S1134DF875FF034C2368002BE4D110BD44C0004068
S1134E0840C00040054B4FF0007210B51A60FEF721
S1134E18A9FD00F043FDFEF7ADFD10BD04ED00E073
S1134E28064B10B5D3F840412388038013B941F2E7
S1134E387B23038000F026FD208010BDA001002004
S1134E4813B5474B47490DF10602C3F840210A68D8
S1134E58454B02EA030343F0E07343F438630B6001
S1134E68424B1B6813F0400FFAD03E4A136823F4F0
S1134E78006313603E4B4FF000521A603D4BD36001
S1134E883D4B13613D4B53613D4B93613D4B136364
S1134E983D4B93603D4B93633D4BD36240323D4B56
S1134EA813603D4B9A4201D00432F8E7FFF702FE43
S1134EB83A4A3B49136843F040031360C03A136805
S1134EC823F040031360B832136843F008031360F7
S1134ED8C03A136823F008031360324B4FF480720E
S1134EE80B60314B1A60314AA3F583631A60304A68
S1134EF802231360013313602E4B00221A600A60E8
S1134F08FDF7A4F82C4B31221A602C4B1C6874B999
S1134F182B482C4900F036FC2B48052200F14001AF
S1134F2800F0A6FD00F06AFD04460028FAD02268C5
S1134F380AB9244905E0254B18689047014600281A
S1134F48E6D0606800F01EFCA068E168052200F065
S1134F588FFD00F053FD04460028FAD0E7E7C04669
S1134F68A001002060E00F400FD43FF850E00F404C
S1134F7808ED00E0814A0000854A0000894A0000E3
S1134F888D4A0000914A0000954A0000994A0000A1
S1134F989D4A0000A14A0000EC00002008E10F40EF
S1134FA8000C004051E5CC1A1804004060343C025F
S1134FB8080000400C00004040E10F4004030020BA
S1134FC86A7B000078030020747B0000080300203B
S1134FD837B5084B01380D46C0B219680401631887
S1134FE81B7B009064581846114602232A46A047A2
S1134FF83EBDC046E402002037B5064B0138C0B2B6
S11350081C6805012B191B7B00902C591846042396
S1135018A0473EBDE402002013B5074B01381A68C7
S1135028C0B201018B181B7B00908C5800211846D4
S11350380A460523A0471CBDE402002073B5084BAB
S11350480138C0B21C6805012B191B7B0E46009061
S113505811462C59184632460723A0477CBDC04642
S1135068E402002037B5074B0138C0B21C680501BB
S11350782B191B7B00900A462C591846002106233D
S1135088A0473EBDE402002037B5084B01380D4661
S1135098C0B21968040163181B7B00906458184651
S11350A811460A232A46A0473EBDC046E402002012
S11350B800B50D4B4FF0000E1A6893F804C00EE0CB
S11350C81368834206D1137B8B4203D10EF101038B
S11350D8D8B207E00EF101035FFA83FE1032E64509
S11350E8EED1002000BDC046E402002011F0100FEC
S11350F810B58646104602D0202300F8013B11F073
S1135108800F06D00346302203F8012B4832427040
S1135118581C01F00703042B28BF042301F02004C2
S11351285A0010E0531EDAB293002EFA03F303F088
S11351380F033033392B04D90CB1073301E027337B
S1135148DBB200F8013B002AECD111F0080F06D0BD
S113515803460D3203F8012B0A224270581C11F041
S1135168400308BF037010BD00E001300378202B12
S1135178FBD0002209E0303BDBB2092B02D9273BE4
S113518803F00F03013043EA021203782F2BF2D8FD
S113519810467047002205E0303B03EB420303EB63
S11351A8C202013003782F2BF6D810467047C04648
S11351B8002301E019540133013AFBD27047C04679
S11351C800B54FF0000E05E01EF801300EF800306F
S11351D80EF1010E013AF7D200BDC04600B54FF0FA
S11351E8000C964609E01CF800201CF801300CF16C
S11351F8010C9A4201D0012003E0BEF1010EF2D263
S1135208002000BD02780B789A4201D0012008E002
S113521810F8013F0131002BF4D10B78181E18BF88
S1135228012070470B7800F8013B11F8013B002B73
S1135238F8D101387047C0460246002000E001302A
S1135248835C002BFBD170472DE9F04104461646D8
S11352588846FEF787FB228A618AB3188B4201DDF0
S11352688B1A9EB2A768E368BA199A42A26001D25F
S1135278354605E0531A2268A3609B1AF31A9DB2B7
S1135288FEF778FB39462A4603E098F8003001F81F
S1135298013C531E9AB24FF6FF7301319A42F4D17E
S11352A8AE420ED0731B9AB2216803E098F800301E
S11352B801F8013C531E9AB24FF6FF7301319A422A
S11352C8F4D1FEF74FFB238AF3182382FEF752FB2F
S11352D83046BDE8F081C0462DE9F0410546164642
S11352E88846FEF73FFB2A8A698AB3188B4201DD98
S11352F88B1A9EB2AF68EB68BA199A42AA6001D2B7
S1135308344605E0531A2A68AB609B1AF31A9CB218
S1135318FEF730FB384641462246FFF751FFA642C6
S113532805D0286808EB0401321BFFF749FFFEF794
S113533819FB2B8AF3182B82FEF71CFB3046BDE8B9
S1135348F081C046038A2DE9F0479A4234BF90465B
S1135358984604460E464768B8F1000F26D0C2683E
S113536807EB08039342436012D3D31B9DB203682F
S1135378C5EB08094B444360FEF7FCFA86B139468D
S11353882A463046FFF71CFF701921684A4605E093
S1135398FEF7F0FA26B1304639464246FFF710FFC9
S11353A8FEF7E0FA238AC8EB03032382FEF7E2FA46
S11353B84046BDE8F087C0462DE9F0411C460E463C
S11353C817469DF81850FEF7CDFA052C04D0062C84
S11353D813D0042C07D01BE0104B1B6803EB0513F8
S11353E85B681C8A15E00D4B31461B683A4603EB93
S11353F805135868FFF7A6FF0EE0084B1B6803EB7C
S113540805135B681A689A605A604FF000021A82A2
S11354180024FEF7AFFA2046BDE8F081E40200203C
S11354282DE9F3410E469046044600285AD1002A35
S113543830D10A784B789A4251D1FEF793FA324D1B
S1135448B17832486971FFF733FEA87160B12B68EF
S1135458327903EB001353F80C0C018A4B1D9B188B
S1135468428A934203DDAC71FEF784FA35E08B1D62
S1135478038206210AE08368327803F8012BC268A4
S11354888360934224BF0368836001360139F2D2F2
S1135498062025E01C4B9D7965B90A784B789A4219
S11354A81DD18C7819482146FFF702FE0546B0B194
S11354B8274603E098715F79FEF75CFA124B314690
S11354C81B68424603EB051353F80C0CFFF704FF63
S11354D80421044678B200F067FA204600E0002070
S11354E880B20EE0FF2801D100200AE0064B441EDA
S11354F8E4B21D6826017319187B009474590323B8
S1135508A047BDE8FC81C046E4020020C153000066
S113551810B584464FF0000E08461EF80C301FFAEA
S11355288EF20EF1010E002BF7D10AB9104602E0F3
S11355386146FFF775FF10BD10B5024B1978FFF7E8
S1135548E7FF10BD2C0100201FB50DF1050422460C
S1135558FFF7CCFD2046FFF7EFFF1FBD7FB58E4652
S1135568164612B90DF1030400E014461EF0100F9C
S113557804D0202304F8013B0EF0FB0E1EF0010FAB
S113558805D0002803DA2D23404204F8013B2E49B4
S1135598002523E00A23B1FBF3F10DB126330AE019
S11355A801290AD11EF0020F01D0302303E01EF0B6
S11355B8040F02D0202304F8013B8142EAD8B0FB4F
S11355C8F1F3DBB203F1300201FB13000A230029D3
S11355D818BF012504F8012BB1FBF3F10028ECD125
S11355E8224605E00A23B1FBF3F1263302F8013C15
S11355F8104619B10132002DF4D100E06DB91EF046
S1135608040F01D0202306E01EF0020F02D030233D
S113561800F8013B302300F8013B1EF0080F06D0C8
S113562803460D2203F8012B0A224270581C1EF06F
S1135638400308BF037026B90DF10300FFF77CFF90
S1135648304604B070BDC04600CA9A3B13B5002466
S11356588DF804008DF8051001238DF807202046E5
S11356680DF1020106228DF802408DF803408DF8F1
S11356780630FFF7D5FE1CBD07B5034680B10020F0
S11356888DF805308DF8071001230DF1030105226B
S11356988DF803008DF804008DF80630FFF7C0FE7E
S11356A80EBDC04670B5044608460D4600F0CAF85B
S11356B828B1431920606060A060E360658270BD12
S11356C82DE9F04705461046894690461E46FFF7E1
S11356D8EFFC014620BBFFF7EBFC0746F0B1124B89
S11356E81B68103B03EB00142B8843B1304600F0D1
S11356F8A9F8606018B12988FFF7D4FF80B16B88D6
S113570843B1304600F09EF8A06018B16988FFF7ED
S1135718C9FF28B1C4F8008084F80C90384600E02A
S11357280020BDE8F087C046E4020020032807B53E
S113573804D0082815D080B1002015E0138901A8E9
S1135748ADF804304FF00003ADF806301368074A8B
S113575819781423FFF7B4FF06E0104600F0EEFBB7
S113576802E0104600F0E2FD0EBDC046C153000041
S113577810B5034C2071000100F064F8206010BDDE
S1135788E40200200E4B4FF000021A805960996021
S11357980C4B82B01A7801E07BB104300378934251
S11357A8FAD14388C818064B986002E0552300F8DC
S11357B8013B0DF107039842F8D902B07047C0467F
S11357C8EC02002004010020044B996800228B1885
S11357D85B7890B20132552BF9D07047EC02002067
S11357E8024B98685B68C01A80B27047EC020020CC
S11357F8034B98685A681B88801AC01A80B270478D
S1135808EC02002070B50E4E0546338872689C1869
S11358184B1E234202D04B4223405C18B3686219E2
S11358289A4201D3002009E0204600212A46FFF7C6
S1135838BFFC73682046EB1A1B19338070BDC04641
S1135848EC02002070B50E4E054673683288D418F1
S113585814F0030F1CBF24F003031C1DB3682218A3
S11358689A4201D3002009E0204600212A46FFF786
S11358789FFC73682046EB1A1B19338070BDC04621
S1135888EC020020044B1B8843F3000000F434406E
S113589880EA53007047C046F8020020134B144AAC
S11358A859681368581C1060F1B118E011F8033CEA
S11358B8ABB151F8083C984211D1D37B022B04D0E8
S11358C80423D37311F8043C137492892AB151F850
S11358D8083C9B1841F8083C01E001F8032C0C3102
S11358E851F80C2C002AE1D17047C046F802002078
S11358F86C0300200F4B70B55C68D4B19D6815E04B
S11359081B7883420DD010E09D4209D1FEF72AF896
S11359180023237263720233EB73FEF72BF808E05B
S11359280C342368002BEFD103E014352B68002BCB
S1135938E6D170BDF8020020194B2DE9F0415D68ED
S11359480E461746002D28D09C6823E01B78834216
S11359581BD01EE09C4217D1FEF704F8E37B23F02A
S11359680203E3732F721FB9A68126B96E7208E089
S1135978002E08BF01260B4B1B68F3186B6001232C
S11359886B72FDF7F7FF08E00C352B68002BE1D1AB
S113599803E014342368002BD8D1BDE8F081C04655
S11359A8F80200206C030020124B70B50E465C68A8
S11359B89D681BE01B78834217D186B964B90EE051
S11359C89D4208D1FDF7CEFF0B4AAB8912689B189C
S11359D86360012304E00C342368002BF0D1002316
S11359E8EE7333B1FDF7C6FF03E014352B68002BC3
S11359F8E0D170BDF80200206C0300201B4B37B5C2
S1135A089D682CE0EB7B13F0050F27D0FDF7AAFF68
S1135A18AB891BB9EB7B13F0010F1AD12A7C9AB11D
S1135A2800248DF803408DF804402B6820461B7829
S1135A380DF103018DF8072005228DF805308DF846
S1135A480640FFF7EDFC2C74EB7B13F0020308BF50
S1135A58EB73FDF78FFF6B682846984714352B685E
S1135A68002BCFD1014BD8683EBDC046F8020020B8
S1135A782DE9F84F9346544A002353609360534BDF
S1135A8882461A780C4645E043B293423DD100233E
S1135A9814F9015F5FFA83F80133002DF8D114205B
S1135AA808FB00F00430FFF7CDFE474BA946986089
S1135AB8631EC8EB03062F4622E054461CE02A78EE
S1135AC84BB29A4217D16368056043602389038106
S1135AD81BB109F101035FFA83F963894381A3893F
S1135AE88381A37BC37343890BB983890BB17B1C63
S1135AF8DFB2143003E010342568002DDFD10136FD
S1135B0871780029D9D101600AE014F9013F002B0A
S1135B18FBD1013420780028B6D180460746814657
S1135B28294CA368002B42D037B30C2307FB03F599
S1135B38281D80B2FFF786FEA16817E04A893AB1AA
S1135B484FF6FF739A4204BF00234B814B8903E04D
S1135B588B890BB91A4601E04360012243680BB1F3
S1135B68012343720AB140F80C1B14310B68002B53
S1135B78E4D1154B421B5A6009EB0B00C0B2FFF786
S1135B88F7FDB9F1000F12D00F4B9C680CE0238984
S1135B984BB1032001212246FFF7C8FDA07310B9B9
S1135BA84FF0FF33A37314342368002BEFD1064D51
S1135BB800242846FFF734F9054B1C60FDF7E4FE82
S1135BC8EC604046BDE8F88FF8020020040100208C
S1135BD86C03002073B591F82820064612F0030FD1
S1135BE80C4613D012F0010F01D0112100E013214B
S1135BF8FDF780FFC0B200286DD194F8283043F037
S1135C08400323F0030384F8283064E012F0200EE4
S1135C185FD10D8B25B922F0400381F8283058E074
S1135C28CB681978636A13F4806F19D012F0040FE3
S1135C3805D022F0040384F82830754611E094F85E
S1135C482A00884205D094F829308B4208D1012DC6
S1135C5806D042F0040384F828300146012500E008
S1135C6800253046FDF746FF23680133236094F886
S1135C78283043F0400384F8283065BBE368626940
S1135C8801339342E36024BFA368E360238B013BA1
S1135C989AB2114B228353F82630588C94F82B303F
S1135CA8CBB1824217D88DF8053001238DF8063020
S1135CB828466FF020030DF1030105228DF80350E7
S1135CC88DF804508DF80730FFF7AAFB84F82B50A1
S1135CD801E0FDF70DFF7CBD0C030020034B10B55C
S1135CE803EB8003D968FFF775FF10BD0C03002090
S1135CF810B50A4B03EB8003DA6892F8283039B1FF
S1135D0823F0200382F828301146FFF763FF03E0ED
S1135D1843F0200382F8283010BDC0460C0300204D
S1135D287A4B2DE9F04153F821400F4603EB8103E8
S1135D38616A064611F4006FDD6812D094F82820D1
S1135D4812F0040F04D022F0040384F828300FE082
S1135D5894F82A30834204D142F0040384F82830AA
S1135D68D2E011F0800F03D094F82930B34202D066
S1135D784FF0000801E04FF00108636A13F0200FA8
S1135D881CD0132E09D195F8283043F0200385F848
S1135D9828306B6801336B60B6E0112E0ED195F88C
S1135DA8283013F0200F00F0AF8023F0200385F88B
S1135DB8283038462946FFF70DFFA5E0236801334C
S1135DC82360636A13F4805F19D02A8B6B8B9A4221
S1135DD80CD82B691E702B696A69013393422B61B5
S1135DE824BFAB682B612B8B01332B8395F82830A8
S1135DF813F0600F03D138462946FFF7EBFEB8F1DC
S1135E08000F45D1228B638B93420ED9531C2383F5
S1135E18E38B0133E38323691E70236962690133C9
S1135E289342236124BFA3682361616A11F0600F60
S1135E3826D094F8283013F0100F21D1228B238C0C
S1135E489A421DD311F0200F0AD095F8283038460D
S1135E5843F0020385F828302946FFF7BBFE06E025
S1135E6838464FF400714FF40052FDF76FFE94F872
S1135E78283043F0100384F82830636801336360E2
S1135E88626A48F2800302EA0303002B3CD134E03F
S1135E98636A13F4807F1DD0E28B002A2DD0A38B74
S1135EA80233A38323699A1A511E62690133934208
S1135EB8236124BFA3682361A36899423CBF638B11
S1135EC8C918E38B0B70238B013323834FF0000332
S1135ED8E38312E0A38B228B0133A383638B934266
S1135EE80BD9531C238323691E7023696269013308
S1135EF89342236124BFA368236194F82B0018B14B
S1135F0840B20421FFF750FDBDE8F0810C030020E6
S1135F1870B505462C20FFF795FC58B10446284671
S1135F28FFF790FCA06028B143192061E060636129
S1135F38658300E00024204670BDC0462DE9F04189
S1135F4805460E463C48297AFFF7B2F8074618B1C9
S1135F5816F0040F06D16CE00146FFF7A9F80746CE
S1135F68002866D0354B344A1B683901103B16F0BB
S1135F78020F03EB01085A5009D0E8882C7AFFF77E
S1135F88C7FF2F4BC8F8080003EB8403D86016F04A
S1135F98010F12D0A888FFF7BBFF2B7A284AC8F84C
S1135FA8040042F823002B6813F4807F05D00369AA
S1135FB8013303614FF001030383214C2B7A04EB73
S1135FC88303DA680AB12B6853622B7A54F82320C6
S1135FD842B32B7B642082F82B302B7AAA8854F89E
S1135FE823106B7B03FB02F393FBF0F30B842B7AF4
S1135FF8AA8854F82310AB7B03FB02F393FBF0F35A
S11360084B842B7A54F823202B6853622B7A54F848
S113601823206B7A82F829302B7A54F82320AB7A20
S113602882F82A302B7A294688F80C30287AFDF72A
S11360380FFE3846BDE8F0814D600000E402002000
S11360480C0300202DE9F0471C46023C80460F460D
S113605816469DF82050FDF785FC082C00F2608157
S1136068DFE814F009008500AB00710019015E0136
S11360785E015E01F10017F4805FA8494FEA051438
S113608803D00B68E3189C6802E00B68E3185C68AB
S1136098002E56D016F0800F05D040463146626A6D
S11360A8FDF754FD4DE016F4806F0BD03146626A5B
S11360B84046FEF77DFC0446C4F300214046FFF742
S11360C817FE2EE116F0010F03D04046FDF7D0FC71
S11360D805E016F0020F02D04046FDF7DDFC16F08D
S11360E8040F03D04046FDF7E3FC05E016F0080F63
S11360F802D04046FDF7F0FC16F0100F03D0636A97
S113610843F4805305E016F0200F03D0636A23F4A8
S11361188053636216F4006F05D0636A84F82970AB
S113612843F4C07305E016F4805F03D0636A23F474
S1136138C073636216F0400F1CBF07F07F0384F836
S11361482B30A48CEDE0754B1B6803EB05135868E2
S1136158436A13F0800F08D013F4807F808B02D039
S1136168431C5C08DDE00446DBE0048BD9E06B4BA0
S11361781B6803EB05139C683FB9628B238BD01A09
S1136188B042C0F2CD8084B2CBE0FDF7F3FB3946D0
S1136198324604F10800FFF79FF80546FDF7E2FBD5
S11361A894F8283013F0600F03D140462146FFF7D6
S11361B811FDFDF7DFFB2846B6E0584B4FEA0519F9
S11361C81B684B445D6848F280136A6A02EA030359
S11361D82BB1AC8B002C00F0A480631EAB8305F1BB
S11361E8080039463246FFF7ADF80446686A10F0ED
S11361F8600F00F0988095F8281011F0100F00F047
S113620892802A8B6B8C9A4200F28D8021F01003C5
S113621810F0200F85F828300DD0404B40461B68FD
S11362284B44996891F8283043F0010381F82830E9
S1136238FFF7D0FC77E040464FF480714FF40052EA
S1136248FDF784FC6FE0012E34494FEA051405D9A3
S11362580B68E3189968B31E9EB202E00B68E31852
S113626859687FB9012E09D92C4B0F601B684F6000
S113627803EB05135B681F605F6001E041F826705B
S11362883C464EE001EB86010020435CC3550130D7
S11362980428FAD144E021492C011EB10B68E31803
S11362A89A6827E00B681B195A6892F8283013F08B
S11362B8100F1FD023F0100382F828300B681B1925
S11362C899684B6A13F0200F09D091F8283040469A
S11362D843F0010381F82830FFF77CFC06E04046D0
S11362E84FF480714FF40052FDF730FC0B4B1B68E0
S11362F81B195A6891684FF000031161D160138328
S113630893836EB9536A13F4807F09D04B1C1361CD
S11363184FF00103D6831383344602E0E4020020DD
S11363280024FDF727FB2046BDE8F08770B5C17946
S11363380446022934D81B48FEF7BAFE0146002851
S11363482ED1FEF7B5FE054650B3A01CE179154AD7
S11363581C23FFF7B5F918B36B1E134DDEB22B6877
S113636830011B185A681149E37941F8232022B1F6
S1136378E37951F82320A37913762B680C491B1869
S11363889A68E37941F8232022B1E37951F823206C
S1136398A37913762046FDF7E9FD731CD8B200E013
S11363A8002070BDBD630000E40200202403002027
S11363B8700300202DE9F0411C4680460F4616461E
S11363C89DF81850FDF7CEFA042C0ED0052C02D0F7
S11363D8032C2BD062E0344B1B6803EB051358687D
S11363E8838A002B5AD0058A59E02F4B2A0186B993
S11363F81B68D3189C68FDF7BDFA0322394620466A
S1136408FEF76AFF0546FDF7ADFAE37D13F0400F8A
S11364183EE01B68D3185868838A002B3ED0013BA2
S1136428838239463246FEF78DFF3BE0002E35D095
S11364381D4B1B6803EB05139C68A16897B9626838
S1136448914203D9638A8A1A9B1A01E002D2531A29
S113645898B202E0238A0BBB608AB0421ED9831B20
S11364689DB21CE0731E01F8013BE368A1609942E8
S113647824BF2368A360FDF77DFA394632462046D7
S1136488FEF72AFF0546FDF76DFAE37D13F0E00FEA
S113649805D120464146FDF7EDFD00E00025FDF756
S11364A869FA2846BDE8F081E4020020402802D8B1
S11364B8A0F1300305E0602894BFA0F13703A0F1F0
S11364C83D03D8B27047C046014B18607047C046B8
S11364D82C0300204FF4CA31002201E001F5806149
S11364E8D3B201328142F9D9092B01D8303304E0FF
S11364F8232B01D8373300E03D33D8B27047C04668
S1136508F7B50B4F0546786880B102AC44F8040D22
S11365180122281D0026FDF79FFC7E60284621469F
S11365280422FDF799FC00B101960198FEBDC0460E
S11365382C030020134B37B50446186850B106E005
S113654883689C4202D1C068D8B903E0103003685C
S1136558002BF5D10025204601A904220195FEF758
S113656873FB019B13B94FF480600AE0B3F1FF3F5A
S113657801D1284605E0044A121B9A4238BF019209
S113658801983EBD2C030020FBFF03002DE9F041D8
S113659807460D4690461E46FFF7CCFF044650B109
S11365A8441B08D0B44228BF344678190530414604
S11365B82246FEF749FB2046BDE8F08170B50D463A
S11365C81646044610B94FF4C83409E0FFF7B2FF81
S11365D8043020F47E7020F0070000F58060241851
S11365E80B4B9C4203D900232B601C460DE020462C
S11365F8FFF7A0FF286028B1201D31460122FEF7CD
S113660823FB02E004F58064EAE7204670BDC04637
S1136618FEFF03000A4B10B51A6842B90AE09368F2
S1136628984203D1137900200B7008E010321368E4
S1136638002BF4D104300122FEF706FB012010BD23
S11366482C03002010B5FDF7EDFB002814BF4FF014
S1136658FF30002010BDC0462DE9F341304B0446FD
S1136668884617460AB9586858E0586848BB651DF3
S11366789D6069460DF10702FFF7A0FF0446002854
S113668841D0009B03F58063043323F47E7121F029
S11366980701A542009109D363189D4206D22046FA
S11366A8FFF7D0FF009BBB422DD2ED182046694668
S11366B80DF10702FFF782FF044620B3A842E0D990
S11366C821E09B681918A1F5C833C3F38F22013B55
S11366D8DB19C3F38F259B2D13D99B2A1ED8C1F52B
S11366E880279B250DE0561CB30203F5C8342046C9
S11366F8FFF720FF014618B120460431FFF7A2FF37
S1136708B2B2AA42EFD1064C4146A36860683A4641
S11367181818FDF7A1FB6368F8186060BDE8FC81F0
S11367282C0300200D4B70B51C6805465CB107E0CE
S1136738284600F077F810B1A06868B903E010346F
S113674821680029F4D12878FFF7B0FE9B2828BFD8
S11367589B20800200F5C83070BDC0462C03002081
S1136768022810B504D003280FD0012817D10DE052
S11367780020FEF78DFA90B16FEA406000216FEABD
S11367885060C0B20A460B4606E00020FEF780FAC5
S113679828B1002201211346FDF78EFB01E04FF0DA
S11367A8FF3010BD70B5044601200D461646FEF7AD
S11367B86FFA034638B9FEF76BFA002808BF412080
S11367C880F00300C3B214F4004F06D06FEA4363A9
S11367D86FEA5363DBB283F0030361041846490C80
S11367E82A463346FDF768FB70BDC04610F4004FD7
S11367F870B504460D46164601D1012002E0440452
S1136808640C0020FEF744FA08B9013804E0214674
S11368182A463346FEF720FA70BDC04610B5FDF788
S113682893F810BD00B5844600220EE012F80CE07F
S11368389E4509D0602B01D9203B02E0402B09D9A1
S11368482033DBB29E4505D10132535C90B2002B54
S10B6858ECD100E0002000BDBA
S1136860C66D000007000000006900007E040000FF
S11368700000000000000000000000000000000014
S11368801800000000000000C0A80003FFFFFF0084
S1136890C0A80001C0A8000108007800202017004B
S11368A05D0A0000000041444D494E00202075540B
S11368B061736B657226755461736B6572204E75D6
S11368C06D6265722031000000000050140406005F
S11368D00000436F6E6E656374696F6E2074696D3A
S11368E06564206F75740D0A00436F6D6D616E648D
S11368F0206C696E6520626C6F636B65640D0A00C1
S113690000000100010010100000010020006804D4
S11369100000160000002800000010000000200005
S11369200000010020000000000000100000000032
S113693000000000000000000000000000002165CD
S1136940F25F2065F1EF2065F2EF2165F22F000080
S11369500000000000000000000000000000000033
S11369600000000000000000000000000000000023
S1136970000000000000000000000000000020658E
S1136980F2CF2065F1FF2165F2FF2065F2FF20655B
S1136990F1AF2166F20F00000000000000000000CB
S11369A000000000000000000000000000000000E3
S11369B000000000000000000000000000000000D3
S11369C000002165F24F2065F2EF2065F1FF20659C
S11369D0F2CF2166F20F0CC1FF3F0000000000005F
S11369E000000000000000000000000000000000A3
S11369F00000000000000000000000000000000093
S1136A000000000000002165F20F2065F22F0CC287
S1136A10FF4F0BC1FFEF0BC1FFFF0CC1FFEF0BC119
S1136A20FF2F000000000000000000000000000034
S1136A300000000000000000000000000000000052
S1136A400000000000002065F15F2065F1DF16936F
S1136A50F85F0BC1FFCF0BC1FFFF0BC1FFFF0BC1E1
S1136A60FFFF0BC1FF9F00000000000000000000BA
S1136A700000000000000000000000000000000012
S1136A8000002165F29F2065F1FF2065F1FF20657C
S1136A90F1FF2165F2AF0FB2FC5F0BC1FFEF0BC139
S1136AA0FFCF11AAFB3F2165F29F2065F25F000032
S1136AB000000000000000000000000000000000D2
S1136AC00000000000002165F24F2165F2EF20650F
S1136AD0F1FF2065F1FF2065F1CF00000000216582
S1136AE0F21F2065F2FF2065F1FF2065F1FF2065AC
S1136AF0F1CF2165F22F000000000000000000002B
S1136B0000000000000000000000000000002165FB
S1136B10F29F2166F22F0CC2FF5F0BC1FFEF0BC186
S1136B20FFEF1693F85F2165F2CF2065F1FF206532
S1136B30F2FF2065F1FF2065F22F00000000000045
S1136B400000000000000000000000000000000041
S1136B5000000BC1FF0F0BC1FFCF0BC1FFFF0BC127
S1136B60FFFF0CC1FFFF0CC1FFAF1D72F36F216566
S1136B70F29F2165F20F00000000000000000000F9
S1136B800000000000000000000000000000000001
S1136B90000000000000000000000CC1FF4F0CC109
S1136BA0FFEF0BC1FFFF0BC1FFCF1693F81F20654A
S1136BB0F23F0000000000000000000000000000A0
S1136BC000000000000000000000000000000000C1
S1136BD000000000000000000000000000000CC1E4
S1136BE0FF0F0CC1FF2F2065F28F2165F2FF206596
S1136BF0F1FF2165F2EF2065F12F00000000000095
S1136C000000000000000000000000000000000080
S1136C1000000000000000000000000000000BC1A4
S1136C20FF5F0BC1FFEF1693F85F2065F1CF20657E
S1136C30F1FF2065F2FF2065F1FF2065F1CF000030
S1136C400000000000000000000000000000000040
S1136C500000000000002065F23F0CC2FF9F0BC142
S1136C60FFFF0BC1FFFF0BC1FFFF0BC1FFAF1D7483
S1136C70F45F2165F2EF2165F29F2165F20F0000B8
S1136C80000000000000000000000000000020657B
S1136C90F14F2165F2EF2065F2FF2065F1CF0FB1CE
S1136CA0FC5F0BC1FFEF0BC1FFFF0BC1FFFF0BC16B
S1136CB0FF9F000000000000000000000000000032
S1136CC0000000000000000000000000000020653B
S1136CD0F12F2065F1EF2065F1FF2065F1FF2065BC
S1136CE0F1FF2165F29F0CC1FF9F0CC2FF2F000032
S1136CF00000000000000000000000000000000090
S1136D00000000000000000000000000000000007F
S1136D100000000000002165F25F2065F1FF21659D
S1136D20F2CF2165F22F00000000000000000000F7
S1136D3000000000000000000000000000000FFF41
S1136D40000003FF000081FF0000C07F0000C03F7F
S1136D500000800F0000C1030000F0010000F803F0
S1136D600000FE070000FF010000FF000000FC001F
S1136D700000F0070000F00F0000FC3F00000000DE
S1136D800D0A0A48656C6C6F2C20776F726C642E48
S1136D902E2E204C4D5331393638204556414C0D5A
S1136DA00A004144432056616C7565733A0D0A002C
S1136DB03D3D3D3D3D3D3D3D3D3D3D000D0A536165
S1136DC06D706C652D0066617669636F6E2E696304
S1136DD06F000000B46E00000F070000467500004D
S1136DE0086F0000140E000055750000B06F00001D
S1136DF0160C000068750000407000000F080000C9
S1136E007A750000A0700000110C00008D75000060
S1136E1030710000110700009C7500003330300011
S1136E200000003630300000000031323030000005
S1136E300032343030000000343830300000003983
S1136E403630300000003134343030000031393213
S1136E5030300000333834303000003537363030CD
S1136E6000003131353230300032333034303000CC
S1136E704F444400004556454E004E4F4E450031A8
S1136E80000000312E3500320000004E4F4E450008
S1136E900000005254530000000000584F4E000000
S1136EA00000000820080000AB750000000000008E
S1136EB004090000AF750000B17500000004000073
S1136EC0C9750000CB75000000050000E6750000E0
S1136ED0E875000000060000F7750000F975000071
S1136EE0000700001376000015760000000900007A
S1136EF04A76000034760000000000004F7600005F
S1136F005476000002000000677600006A760000F4
S1136F10000D00007A76000083760000070100006F
S1136F2099760000A476000004010000B376000006
S1136F30BF76000004020000D2760000DE76000076
S1136F4004030000F276000000770000040600004D
S1136F501C77000028770000040500004377000038
S1136F6051770000040A0000757700007A7700006A
S1136F7003060000967700009F77000003050000D9
S1136F80C3770000CA77000004070000DC77000024
S1136F90E3770000040800004A760000347600001D
S1136FA0000000004F76000054760000020000004C
S1136FB0677600006A760000000D0000F477000098
S1136FC0FD77000005000000127800001B78000027
S1136FD005010000337800003C7800000502000041
S1136FE05078000058780000050300007378000012
S1136FF07C780000050400009C780000AB78000059
S113700005150000C6780000D478000005160000BD
S11370101C770000F178000005110000757700006E
S11370207A770000030600004A76000034760000F8
S1137030000000004F7600005476000002000000BB
S1137040677600006A760000000D00000B790000EE
S11370501379000001020000317900003979000041
S1137060010B0000537900005D7900000104000069
S1137070747900007F790000010500007577000035
S11370809C790000010C00004A7600003476000070
S1137090000000004F76000054760000020000005B
S11370A0677600006A760000000D0000B9790000E0
S11370B0C179000007020000DD790000E8790000D2
S11370C007000000087A0000107A0000070300009F
S11370D02C7A0000397A0000070500001C770000B4
S11370E0647A000006020000757700007A770000D9
S11370F003060000777A00007E7A00000307000090
S1137100967A00009E7A000003020000B77A00001D
S1137110BD7A0000010000004A76000034760000C9
S1137120000000004F7600005476000002000000CA
S1137130677600006A760000000D0000E57A000022
S1137140CA7A000004040000E37A0000EC7A00002C
S1137150040B0000067B00000E7B0000010A000007
S1137160227B0000297B0000010100004A76000018
S113717034760000000000004F76000054760000D2
S113718002000000202D2000656E61626C65640DB4
S11371900A0064697361626C65640D0A000A0D5328
S11371A0657269616C206E756D6265723A20005378
S11371B06F6674776172652076657273696F6E208D
S11371C000446576696365206964656E74696669FF
S11371D0636174696F6E3A20000A0A0D000A0D3D5E
S11371E03D3D3D3D3D3D3D3D3D3D3D3D3D3D3D3DCB
S11371F03D3D0A0D00656E61626C650064697361F2
S1137200626C65000D0A496E76616C69642073775F
S1137210697463680D0A000A0D53797374656D20EF
S11372206D656D6F7279207573653A0A0D0046724B
S113723065652068656170203D20002066726F6D71
S113724020000A0D556E7573656420737461636B59
S1137250203D20000D0A54686520646576696365E5
S113726020686173206265656E206F706572617459
S1137270696E6720666F72200042616420706F72CD
S113728074206E756D6265720D0A000D0A506F727E
S11372907420646972656374696F6E3A20004F5597
S11372A0545055540D0A00494E5055540D0A004986
S11372B06E76616C696420706F72740D0A00506F91
S11372C0727420697320696E7075740D0A00506FB2
S11372D072742073746174653A2000310D0A0030B1
S11372E00D0A000D0A3F3F0D0A23000A0D4279657D
S11372F0204279650A0D000A0D506172616D657452
S11373006572207365740A0D000A0D54656D702E44
S113731020506172616D65746572207365740A0D25
S1137320000A0D506172616D657465722076616C3E
S11373307565203D20000A0D4E6F2076616C6964EE
S113734020706172616D6574657273206176616924
S11373506C61626C650A0D000A0D4F726967696E93
S1137360616C20706172616D657465727320726501
S113737073746F7265640A0D000A0D466163746F5D
S1137380727920706172616D6574657273207265C3
S113739073746F7265640A0D000A0D506172616D39
S11373A0657465727320696E76616C696461746575
S11373B0640A0D000A0D4E657720506172616D6597
S11373C0746572732076616C6964617465640A0D16
S11373D0000A0D436F6E66696775726174696F6E3A
S11373E02073617665640A0D00496E636F7272657D
S11373F063742064617461206C656E6774680D0A3F
S1137400000D0A53657269616C20636F6E6669676B
S113741075726174696F6E0D0A0042617564203D76
S11374202000696E76616C696421003700380020A1
S1137430426974730D0A002073746F70206269745A
S11374402873290D0A00466C6F7720636F6E74727F
S11374506F6C20004869676820776174657220004A
S1137460250D0A004C6F7720776174657220000D3A
S11374700A53656375726974792073657474696EEF
S113748067730D0A005465726D696E616C206D65D9
S11374906E75206C6F67696E0054454C4E455420E0
S11374A07365727665720020202054656C6E657475
S11374B020706F7274206E756D626572203D2000BD
S11374C0496E636F72726563742073657269616C6F
S11374D02073706565640D0A00496E636F7272658E
S11374E06374207061726974790D0A00496E636F68
S11374F072726563742073746F7020626974730DA3
S11375000A00496E636F727265637420666C6F77EC
S113751020636F6E74726F6C0D0A000A0D41525035
S1137520207265736F6C7665640A0D000A0D415212
S113753050207265736F6C7574696F6E2066616933
S11375406C65640A0D0020202020204D61696E20A6
S11375506D656E7500204C414E20636F6E666967E1
S113756075726174696F6E002020205365726961C1
S11375706C20636F6E6669672E0020496E707574A7
S11375802F4F7574707574206D656E750020202002
S113759041646D696E2E206D656E75002020205348
S11375A0746174732E206D656E75004D4143003116
S11375B000436F6E666967757265204C414E2069A1
S11375C06E74657266616365003200436F6E66694E
S11375D0677572652073657269616C20696E746584
S11375E07266616365003300476F20746F20492F12
S11375F04F206D656E75003400476F20746F2061F5
S1137600646D696E697374726174696F6E206D65FF
S11376106E75003500476F20746F206F7665727643
S11376206965772F73746174697374696373206D0A
S1137630656E7500446973706C6179206D656E7553
S11376402073706563696669632068656C70007196
S1137650756974004C6561766520636F6D6D616E4C
S113766064206D6F646500757000676F20746F200F
S11376706D61696E206D656E75007365745F646815
S11376806370003C656E61626C652F64697361624E
S11376906C653E2044484350007365745F69705FB5
S11376A061646400536574204950206164647265A8
S11376B07373007365745F69705F6D61736B0053FE
S11376C06574204950207375626E6574206D617312
S11376D06B007365745F69705F67776179005365E8
S11376E0742064656661756C742067617465776184
S11376F079007365745F6574685F737065656400B1
S1137700536574204C414E207370656564202831A4
S1137710302F3130302F4155544F290073686F7723
S11377205F636F6E6669670053686F77206E657478
S1137730776F726B20636F6E6669677572617469C7
S11377406F6E0073686F775F636F6E6669675F6FF4
S11377500053686F77206F726967696E616C206E81
S11377606574776F726B20636F6E6669677572619B
S113777074696F6E0073617665005361766520638A
S11377806F6E66696775726174696F6E20746F20BD
S1137790464C4153480076616C69646174650056D7
S11377A0616C69646174652074656D706F72617277
S11377B07920636F6E6669672E20696E20464C419E
S11377C0534800617270202D6100526571756573B4
S11377D07420415250207461626C650061727020A3
S11377E02D640044656C65746520415250207461B9
S11377F0626C65007365745F6261756400536574DF
S11378002073657269616C206261756420726174B1
S113781065007365745F73746F70005365742073CF
S1137820746F7020626974732028312F312E352FC4
S11378303229007365745F62697473005365742040
S11378406461746120626974732028372F382900B9
S11378507365745F7061720053657420706172693E
S1137860747920284556454E2F4F44442F4E4F4E91
S11378704529007365745F666C6F770053657420E7
S1137880666C6F7720636F6E74726F6C2028584F2C
S11378904E2F5254532F4E4F4E4529007365745F3B
S11378A0686967685F776174657200536574206600
S11378B06C6F77207374616C6C20282529205B31F0
S11378C02E2E39395D007365745F6C6F775F776155
S11378D07465720053657420666C6F7720726573EB
S11378E07461727420282529205B312E2E39395D6C
S11378F00053686F772073657269616C20636F6EE3
S113790066696775726174696F6E007365745F642C
S113791064720053657420706F727420747970659A
S1137920205B312E2E345D205B3C693E7C3C6F3EF7
S1137930006765745F6464720047657420646174F1
S11379406120646972656374696F6E205B312E2EE9
S1137950345D00726561645F706F727400526561BA
S11379606420706F727420696E707574205B312EA0
S11379702E345D0077726974655F706F72740053A2
S1137980657420706F7274206F7574707574205BE9
S1137990312E2E345D205B302F315D0053617665CE
S11379A020706F72742073657474696E67206173DC
S11379B02064656661756C74007365745F667470C9
S11379C0003C656E61626C652F64697361626C650D
S11379D03E20465450207365727665720073657458
S11379E05F74656C6E6574003C656E61626C652FD6
S11379F064697361626C653E2054656C6E657420C5
S1137A0073657276696365007365745F7765620098
S1137A103C656E61626C652F64697361626C653E7E
S1137A202057454220736572766572007365745FF2
S1137A307765625F61757468003C656E61626C6550
S1137A402F64697361626C653E20574542207365FB
S1137A50727665722061757468656E7469636174A9
S1137A60696F6E0053686F7720636F6E6669677520
S1137A70726174696F6E0072656A65637400526541
S1137A80736574206E6F6E2D736176656420636810
S1137A90616E67657300726573746F726500526519
S1137AA073746F726520666163746F727920736595
S1137AB07474696E677300726573657400526573DC
S1137AC06574206465766963650053686F77204543
S1137AD0746865726E657420737461746973746913
S1137AE0637300725F6970737461740052657365C7
S1137AF0742045746865726E65742073746174696A
S1137B0073746963730075705F74696D650053689D
S1137B106F77206F7065726174696E672074696D28
S1137B2065006D656D6F72790053686F77206D65C0
S1137B306D6F7279207573650056312E332E303196
S1137B403100000099430000BD430000E143000000
S1137B5005440000254D0000094D0000ED4C0000D7
S1137B600000000303030880400001005866000081
S1137B7000000000BC7B000025680000000000003D
S1137B8004000100C17B0000252300004500020021
S1137B9000000000C57B00007D3800002500FFFFC9
S1137BA000000000000000000000000000000000D1
S1137BB0000000000157616D4E73000057646F6749
S1137BC000617070006D61696E74656E616365005B
S1137BD048544D004A504700474946004353530018
S1137BE04A530042494E005458540049434F003F01
S1067BF03F3F0010
S1137BF4FF00000001000000D07B0000D47B0000E3
S1137C04D87B0000DC7B0000E07B0000E37B000009
S1107C14E77B0000EB7B0000EF7B0000FF2E
S9032008D4
